:102CD800120100020000004005165F810000010299
:0C2CE80000010A0600020000004001008C
:102CF4000902200001010080F00904000002FF0025
:102D04000000070502020002000705860200020017
:102D14000902200001010080F00904000002FF0004
:102D2400000007050202400000070586024000007B
:102D3400040309040C03410043004300450053000D
:102D440026035500530042002D0041004900200095
:102D540020002000200020002000200000000000AF
:082D6400000000000000000067
:102301006080E000013F01010101010700030202B9
:1023110002020200F5F7F7F7F7F7F7F70000000000
:102321000000003F013F010101010107020500001A
:1023310000000000F6F7F7F7F7F7F7F700000000E5
:102341000000003F011301210139010700010001D3
:10235100000B0200FFFFFBFFFDFFFFF7003600F05F
:102361000012003F010138010101010702020D00C5
:1023710000000000F2F7F7F7F7F7F7F700002D007C
:102381000000003F6024E087000000000000000022
:10239100000000000000000000000000000000003C
:1023A10000000000000000000000000047E080E0A5
:1023B1008000F7AA4E006080E0AB013F01010101FE
:1023C10001070003020202020200F5F7F7F7F7F72F
:1023D100F7F7000000000000003F013F010101018B
:1023E10001070205000000000000F6F7F7F7F7F714
:1023F100F7F7000000000000003F0113012101393F
:10240100010700010001000B0200FFFFFBFFFDFFC0
:10241100FFF7003600F0002D003F010138010101F6
:10242100010702020D0000000000F2F7F7F7F7F7CD
:10243100F7F700002D000000003F6024E1320000AA
:10244100000000000000000000000000000000008B
:10245100000000000000000000000000000000007B
:0C246100000047E12BE08000F7AA4E00CD
:103CA50090E60174AAF090E6F574FFF022F59B7595
:103CB5009DE4E4F59EFF2290E67BE090E67CF00F24
:013CC50022DC
:102BAE00123CA590E12BE090E6F3F090E12CE09042
:102BBE00E6C3F090E12DE090E6C1F090E12EE090BA
:102BCE00E6C2F090E130E090E6C0F090E131E090A6
:102BDE00E6F4F075AF0774E0F59A74AB123CB212DE
:102BEE003CBCBF80FA000000E490E6C4F000000098
:102BFE0090E6C5F090E132E090E6C6F090E133E069
:102C0E0090E6C7F090E134E090E6C8F090E135E050
:102C1E0090E6C9F090E136E090E6CAF090E137E038
:102C2E0090E6CBF090E138E090E6CCF090E139E020
:042C3E0090E6CDF05F
:012C4200226F
:102C4300123CA590E080E090E6F3F090E081E09004
:102C5300E6C3F090E082E090E6C1F090E083E0907C
:102C6300E6C2F090E085E090E6C0F090E086E09068
:102C7300E6F4F075AF0774E0F59A7400123CB212F3
:102C83003CBCBF80FA000000E490E6C4F000000002
:102C930090E6C5F090E087E090E6C6F090E088E02B
:102CA30090E6C7F090E089E090E6C8F090E08AE013
:102CB30090E6C9F090E08BE090E6CAF090E08CE0FB
:102CC30090E6CBF090E08DE090E6CCF090E08EE0E3
:042CD30090E6CDF0CA
:012CD70022DA
:0A3F21000001020203030404050579
:103AB300EC4EFEED4F2421F582743F3EF583E493F3
:103AC300FF3395E0FEEF24A1FFEE34E68F82F5830A
:103AD3002290E6BCE0547EFF7E00E0D394807C001D
:013AE30022C0
:03000B000231E9D6
:1031E900C0E0C0F0C083C082C085C084C086758637
:1031F90000C0D075D000C000C004C005C006C0071B
:103209000564E564B406270518E51870020517AECC
:1032190017FF7C007D0A12135FED4C700E90E1A33D
:10322900E004F0700690E1A2E004F0756400D007B4
:10323900D006D005D004D000D0D0D086D084D08597
:09324900D082D083D0F0D0E03235
:102DFF00E4F532F531F530F52FC219C216C218C2FB
:102E0F0017121D8875672C7568D8756F2C7570EA49
:102E1F0075652C7566F4756D2D756E1475712D7540
:102E2F007234D2E843D82090E668E04409F090E687
:102E3F005CE0443DF0D2AFD20D123B1590E680E03E
:102E4F0054F7F0538EF8C2193017051224AFC2177A
:102E5F00301929123EC25024C219123C3A201616BC
:102E6F0090E682E030E704E020E1EF90E682E03088
:102E7F00E604E020E0E4123B44123ED41229B8806D
:012E8F00C77B
:1024AF0090E6B9E070030225601470030225B4248E
:1024BF00FE700302260E24FB700302255A147003CC
:1024CF0002255414607314607624056003022645B8
:1024DF00123F76400302265190E6BBE024FE6022B5
:1024EF0014603324FD601114602224067048E567E0
:1024FF0090E6B3F0E5688037E56F90E6B3F0E570EE
:10250F00802DE56990E6B3F0E56A8023E56B90E6F0
:10251F00B3F0E56C801990E6BAE0FF123B70AA06A3
:10252F00A9077B01EA494B600DEE90E6B3F0EF90FF
:10253F00E6B4F002265102264A123F3F02265112FC
:10254F003F35022651123603022651123F2B022627
:10255F0051123F78400302265190E6B8E0247F6085
:10256F00151460192402703AA216E43325E0FFA275
:10257F0018E4334F8018E490E740F08016123AD4F5
:10258F0040047D0180027D00123AB3E0540190E7D0
:10259F0040F0E4A3F090E68AF090E68B7402F0022C
:1025AF00265102264A123F7A400302265190E6B87E
:1025BF00E024FE60162402600302265190E6BAE082
:1025CF00B40105C21602265102264A90E6BAE070FF
:1025DF002C123AD440047D0180027D00123AB3E000
:1025EF0054FEF090E6BCE05480131313541FFFE029
:1025FF00540F2F90E683F0E04420F08045803C128A
:10260F003F7C503E90E6B8E024FE601A2402703200
:10261F0090E6BAE0B40104D216802790E6BAE0B48F
:10262F000202801E8015123AD440047D0180027D83
:10263F0000123AB38008120056500790E6A0E0440B
:09264F0001F090E6A0E04480F0E7
:01265800225F
:0300330002004E7A
:04004E0053D8EF3262
:02246D00C11A92
:103C150090E19EEFF0F5CB8FCDAF0590E19FEFF0F2
:103C2500F5CA8FCCE4F5C8758E19D2BDD2AFD2AD29
:053C3500D2CAF51F22B8
:0D00360090E19EE0FF90E19FE0FD023C158F
:083F4900A21B921CD21BA21C5A
:013F5100224D
:083F5200A21B921DC21BA21D5F
:013F5A002244
:033F7000AF1F225E
:033F7300A21B226C
:103EE600AD07AC06C3E49DFBE49CFFEBFD023C156D
:05002E00C2CAC2AD22B0
:03002B00023D2370
:023D2300C0E0FE
:103D2500301B0E301A04051F8007D21A123F5BC2E2
:093D35001A300303123F5BC2CFF8
:033D3E00D0E032A0
:030043000229008F
:030053000229007F
:10290000023C5F00023CE500023CC600023D0400C0
:102910000232BB0002393A00023F7E00023F7F00D4
:10292000023F8000023F8100023C8300022F1C0016
:1029300002365A00023F82000236B000023F830096
:102940000230A000023F7F00023F8400023F85006A
:102950000233ED00023F860002344600023F87004A
:10296000023F8800023F7F00023F7F00023F7F005E
:10297000023F8900023F8A00023F8B00023F8C0029
:10298000023F8D00023F8E00023F8F00023F900009
:1029900002349F00023F91000234F800023F92008F
:1029A00002355100023F93000235AA00023F940015
:0829B000023F9500023F960072
:103B440090E682E030E004E020E60B90E682E0308C
:103B5400E119E030E71590E680E04401F07F147E3F
:0C3B6400001237F290E680E054FEF022E0
:103C3A0090E682E044C0F090E681F04387010000FC
:043C4A000000002254
:103B1500300D0990E680E0440AF0800790E680E0E9
:103B25004408F07FDC7E051237F290E65D74FFF005
:0F3B350090E65FF05391EF90E680E054F7F022B6
:023B7000A907A3
:103B7200AE71AF728F828E83A3E064037017AD01C2
:103B820019ED7001228F828E83E07C002FFDEC3EC6
:093B9200FEAF0580DF7E007F001C
:013B9B002207
:1037F2008E378F3890E600E054187012E5382401B5
:10380200FFE43537C313F537EF13F538801590E62B
:1038120000E05418FFBF100BE53825E0F538E53716
:1038220033F537E5381538AE37700215374E600577
:06383200123C4E80EE2264
:103C4E007400F58690FDA57C05A3E582458370F989
:013C5E002243
:10198A00253032625800253034580020213D20008D
:10199A000D004020504F535420002D2050415353E6
:1019AA00200D002D204641494C200D00362D3136A0
:1019BA004100362D31364500322D31364100322D67
:1019CA00313600322D31364500362D313646003655
:1019DA002D36344D4100362D36344D4500322D36E4
:1019EA00344D4100322D36344D00322D36344D45BA
:1019FA0000362D33324100362D33324500322D3335
:101A0A00324100322D333200322D33324500362D29
:101A1A0036344100362D36344500322D36344100F5
:101A2A00322D363400322D36344500362D393641C2
:101A3A0000362D39364500322D39364100322D39DE
:101A4A003600322D39364500362D313238410036CE
:101A5A002D3132384500322D3132384100322D31A4
:101A6A00323800322D31323845002D4F5448455214
:101A7A0000210054445F504F4C4C3A20475049468D
:101A8A0054524947202620307838300D005F0056DE
:101A9A0044656320333020323031394031333A31B2
:101AAA00373A34370000475049464D6F64655365ED
:101ABA00743A0020434F4E54494E554F55530D002A
:101ACA002054430D002D2030784243205772697408
:101ADA006520002D205069636B47504946203D2000
:101AEA0000436F6E74696E756F75732000544320DE
:101AFA004D6F646520002D2057726974652034305B
:101B0A003146203D203078002D2054436F756E7485
:101B1A00203D203078002D204144435F436F6E748E
:101B2A00696E756F75733D002D204354525265617D
:101B3A00640D002D204354524D6F646520002D2002
:101B4A004354524C6F6164200D002D204354524D72
:101B5A006F64654C6F616420002D2044494F5772B1
:101B6A00697465416C6C3A002D2044494F5F526597
:101B7A006164416C6C3A002D2044494F5F436F6E9B
:101B8A006669677572653A002D204144435F536563
:101B9A0074436F6E6669673A002D204144435F477C
:101BAA006574436F6E666967002D20307842463A45
:101BBA00476574496D6D6564696174652000537485
:101BCA0061727420312041444320436F6E766572FE
:101BDA0073696F6E200054616B6520322041444363
:101BEA002C206672657368206461746120005461F8
:101BFA006B652031204144432C20686973746F72ED
:101C0A006963616C206461746120002D2053656CE6
:101C1A006620546573743A002D2050415353002DA9
:101C2A00204641494C002D2050726F626520436165
:101C3A006C3A002D20537570706F727465642000C1
:101C4A002D20556E617661696C61626C65002D208C
:101C5A0057726974652043616C200D002E0020754F
:101C6A006E617661696C61626C652E002D20565238
:101C7A005F4E4F5344504155544F002D20444F203E
:101C8A004E4F542057414E54002D2056525F524118
:101C9A004D20262056525F454550524F4D0D002D7E
:101CAA00203078423320444143446972656374208A
:101CBA000D002D2030784233204441434D756C7419
:101CCA00694469726563743A20002D204441434493
:101CDA00697265637420526561643A0025332E3156
:101CEA00662C2025332E3166207C2025332E316642
:101CFA002C2025332E3166207C2025332E31662C6C
:101D0A002025332E3166207C2025332E31662C2067
:101D1A0025332E3166002D20444143536574426FAA
:101D2A0061726452616E6765002D2054445F537579
:101D3A007370656E640D002D2054445F526573758F
:101D4A006D650D002D2052657365740031206F7525
:101D5A0074003220696E6F757400455036696E6F73
:101D6A0075740049424E004E3200706E3600656648
:0E1D7A003200656636004646320046463600A8
:10246F0041E19C0041E1C4FF41E19DFE41E1DD00FE
:10247F0041E1C70042E19A0200C106C101020C000E
:10248F0000C107C109C103C10BC10541E19EFB4159
:0F249F00E19F50C10402080000020A0000C100C2
:10209F00142440F58274E73CF583EFF022E4F54514
:1020AF00AF45054574402FF582E434E7F58322E010
:1020BF00FF0540E540AC3F22E490E68AF090E6BE93
:1020CF00E090E68BF02224A4F58274E13EF583E0E4
:1020DF00FCA3E0FDA3E0FEA3E0227BFFE4F53C754B
:1020EF003D01227BFF753C01753D012290E6BAE070
:1020FF0075F008A4FFA3E07C002FFFEC35F0FEE4A1
:10210F002FF58274503EF583E022AD3C7AE779409B
:10211F007F40AB0722E090E740F0E490E68AF09032
:10212F00E68B22FF90E6BAE075F008A42403F5824F
:10213F00E5F03450F583EFF02290E65BF090E65A2D
:10214F00E04401F090E65974FFF090E658E0441037
:10215F00F02290E6BCE0FF90E6BBE02275860053CC
:10216F0091EF90E65D222538F538E53B3537F537A9
:10217F00C3E53A953CF53AE539953BF5392290E6BA
:10218F00BDE090E6BCFEE07C002400FFEC3E229018
:10219F00401C7401F0E4F0904011F022E54275F01C
:1021AF0002A42444F9742D35F0227440253EF582A3
:1021BF0074E7353DF58322C20890E1D9E0904011D4
:1021CF00F022FE74402FF58274E73EF58322E490EF
:1021DF00E1A2F0A3F0F517F5182290E671F090E662
:1021EF0072F075B4FF75B6FF2274E1F59A745AF563
:1021FF009B74E7F59D74C0F59EE422904017E09024
:10220F00E740F0904018E090E741F0227B017AE13F
:10221F00795A22C3E53E953CE53D953B22E490E695
:10222F008AF090E6BEE022F583E0F8A3E0F9A3E0A0
:10223F00FAA3E0FB228F4A8E498D488C4722AF4A82
:10224F00AE49AD48AC47227BFF753C01E4F53D221A
:10225F0090E6047480F022FFAE45054574402E22AF
:10226F007BFF7A19799A22E53EAE3D780222E53856
:10227F00253EF582E537353DF583225391EF90E604
:10228F005F227C007B002412F9EC3400FA227BFFE2
:10229F00E4F53CF53D22F582E43440F583223EF52A
:1022AF0083E0FBED25E0FFEC3322142440F582742C
:1022BF00E73CF583EF22F582E434E1F583227441A4
:1022CF002FF58274E73EF58322856A82856983A3A1
:1022DF007402F022856C82856B83A37407F022E56C
:1022EF0045AD46FCE4020FE99050037474F074B4EA
:0222FF00F022CB
:05004600A21E9204223D
:1037A800200404E4FEFF2290E6A2E020E1F91222C0
:1037B8001B123E62EF2401F54CE43EF54B1221F852
:1037C800FFFEC3EF954CE54B6480F8EE648098509B
:1037D8000F90E67BE090E67CF00FBF00010E80E2E0
:0937E800E54C90E68FF0AE4BFFBA
:0137F10022B5
:1038BD008B488A49894A200404E4FEFF221238F31A
:1038CD008E518F5285484E85494F854A5012221B85
:1038DD001237061238F3745A2FF58274E13EF583D0
:1038ED00E4F01237A822AB48AA49A94A123E622237
:103E8B00200404E4FEFF2290E15AEFF0E4A3F012C9
:033E9B0037A82223
:103D7D00200404E4FEFF22754BFF754C19754D8A26
:0C3D8D008F4E12221B1215771237A8224D
:103D4100200404E4FEFF22754BFF754C19754D905C
:0E3D51008E4E8F4F12221B1215771237A822AA
:1032520090E685E02405F573200404E4FEFF22785D
:103262005A7CE17D011214FE90E6A2E030E1079063
:06327200E685E0B573F2F1
:1032780012221B123E62EF2401F577E43EF5761226
:1032880021F8F574F575C3E5759577E5766480F8EA
:10329800E574648098501290E67BE090E67CF00537
:1032A80075E57570E1057480DDE57790E68FF0AE21
:0232B80076FF9F
:0132BA0022F1
:1038FD0075440390E1DE7430F0E4A3F0A374031279
:10390D0039277F0F123DB590E1DE7438F0E4A3F056
:0A391D00A3041239277F0F023DB505
:10392700F07AE17BDEAD447F0E123DB57AE17BDEB6
:03393700AD44227A
:062FA5008F448D458B46B0
:102FAB002006061222EE0230131222EEE54475F0D3
:102FBB0008A424A4F582E434E1122236120E65E54E
:102FCB004475F008A424A8F582E434E112223612E9
:102FDB000D74122244E4FBFAF9F8120F6B600940EE
:102FEB0007E4FFFEFDFC800312224D1222447B00FE
:102FFB007AFF797F7847120F6B500A7F007EFF7D37
:10300B007F7C47800312224D12224412224D121054
:0A301B0022AD07AC06AF44023323D8
:043F64004380022272
:043F68005380FD2263
:043F6C00638002224A
:103E9E0012225F0000007406F0000000E4F0000043
:023EAE000022F0
:103E2000C20B90E61474E0F000000090E61A7409EA
:073E3000F0000000023E9EBD
:103EB00012225F0000007402F0000000E4F0000035
:023EC0000022DE
:10387B0090E61274A0F000000090E6187411F000AE
:10388B000000123EB090E6917480F0000000F00052
:10389B000000F0000000F000000090E6497482F098
:1038AB00000000F0000000F0000000F0000000023B
:0238BB003EB01D
:0628FA0012387B023E20B3
:01005200228B
:103D5F00E516FE7C00E42515F50FEC3EF50E450F3C
:0E3D6F007007C28CC2A9C20C22D28CD2A9222B
:103AE4001220CC90E6A0E020E1F9E4FF74422FF527
:103AF40082E434E7F583E0FEEF122291EE12132BF9
:103B04000FBF03E890E740E0F515A3E0F516023D8A
:013B14005F51
:1028380090E6B8E030E7621220ACE515F01220AF60
:10284800E516F0E4F544E544C3940350207E007B8C
:102858000074122544F9EE3400FA1212E5FF7440B0
:1028680025451220B6EFF00544054580D9122267A8
:102878001220B6E518F0E5171222661220B6EFF01E
:10288800A20CE4331222661220B6EFF0C20C12201A
:10289800C790E6A0E04480F0221220CC90E6A0E0A9
:1028A80020E1F9C20C90E6BEE064056004E4F5118D
:1028B800221220ACE0F5151220AFE0F516E4F5443D
:1028C800E544C394035018744025451220B6E0FF30
:1028D800E544122291EF12132B0544054580E112BD
:1028E8003D5F90E6BAE0B4CE08A3E0B4AC031200B2
:0128F800528D
:0128F90022BC
:103E3700E5125403904014F0A3E513F0A3E514F042
:063E47001221DDD20C2265
:0F3EF600D3E518950FE517950E4003123E3722BE
:103E4D00C20C1221DDC28CC2A9538EF75389F143E6
:053E5D008901023D5F38
:10397500E50945086019E50915097002150814C31C
:1039850094FFE508648094805018123F688013E521
:1039950011600F7508057509FF123F64E4F51112F2
:0839A50021DE300C0375110155
:0139AD0022F7
:0F3F0500D20812219E75B3FF75B5FF1221E92274
:0D3F140012219ED208F5B3F5B51221E92265
:10000E0090401C7401F0E4F01221C6E4F5B3F5B58E
:0D001E0090E671F090E672F0F5B4F5B622B0
:103DD10012219E1221C675B3FF75B5FF90E671746D
:0B3DE100FFF090E67274801221F022C7
:073B9C00904010F0123F05FC
:103BA300E4FEFD7801AF05EF08800103D8FDF5B110
:103BB3008DB08EA08E9090401BEEF00EEE70E40D53
:033BC300ED70E0C2
:013BC60022DC
:10311000E4F546F547AF477801EF08800103D8FD95
:10312000F5B18546A090401C7401F085904485B0AF
:1031300045E4F0E544B54606E5456547602B90E17A
:103140009D7401F0AF47123D7DAF46123D7D7BFF80
:103150007A1979951238BDAF45123D7DAF44123DC5
:103160007D12226F1238BD80060546E54670A60521
:0E31700047E54770A090E19DE0B4FE02E4F058
:01317E00222E
:103A19007BFF7A19799C1238BD7401123B9C74059D
:103A2900123B9C123F1412311090E19DE07BFF7014
:103A3900067A1979A480047A1979AD1238BD9040B3
:043A490010E4F02273
:062D6C008B3E8A3F894006
:102D7200E4F541754207123E628F4312211B7D0129
:102D82007F047E0012375890E740E04480902CE3A5
:102D9200F090E740E0B4010C1221AB8982F5837414
:102DA2004FF005421221AB8982F5837431F005425E
:102DB200E543254225E0902D44F0E4F541AF43EF91
:102DC2003395E0FEC3E5419FEE6480F8748098502D
:102DD2002BAB3EAA3FA9408541827583001212FEA9
:102DE200FDE5411221ADFAE54275F002A429F9EAA6
:0C2DF20035F08982F583EDF0054180C1C9
:012DFE0022B2
:103BC70090401374AAF0E064AA70197455F0E06489
:103BD700557011744FF0E0B44F0A7449F0E0B449DE
:073BE700037F00227F012291
:10317F00123BC7EF14601B04705A12211B7D017F95
:10318F00037E0012375890E740E0541F90E1C4F0DF
:10319F00804212211B7D027FF67E1D12375890E769
:1031AF0040E0FF780208800123D8FDF53890E74111
:1031BF00E090E1C4F012211B7D017F037E001237E6
:1031CF005890E740E0653860037F042290E740E0C5
:0931DF00541FFF2290E1C4E0FF3F
:0131E80022C4
:103E770090401AEDF090E1DDE53CF090E1C7E53DBB
:043E8700F0022D6CAC
:1027610012211B7D047FCC7E1D1237587F437E438F
:102771007D417C4490E740E0F8A3E0F9A3E0FAA3AF
:10278100E0FBC31213C27068D20112211B7D207FAE
:10279100D07E1D123758E4F544F545E545AE447841
:1027A10002C333CE33CED8F924401221D5E0FCA3A5
:1027B100E0FDA3E0FEA3E0FFC004C005C006C00722
:1027C100E545AE447802C333CE33CED8F924A4F51F
:1027D1008274E13EF583D007D006D005D0041213F0
:1027E100D30545E545700205446408454470AC22B3
:1027F100C201E4F544F545E545AE447803C333CE63
:1028010033CED8F9FBAA0624A4F58274E13AF58304
:102811001213DF3F80000074A82BF58274E13AF5B2
:10282100831213DF000000000545E54570020544F1
:062831006404454470C17F
:01283700227E
:101D8800E4F537C202904019F090E6017480F01231
:101D9800000390E678E04401F0E05410FFC4540FCB
:101DA800445090E159F0E013E43390E1C6F090E636
:101DB800007410F0123E4D904019E4F090E6107453
:101DC800A0F090E611F000000090E612F00000008C
:101DD800E490E613F000000090E61474E0F00000D0
:101DE80000E490E615F012225F0000007402F00093
:101DF80000007406F0000000E4F000000090E6180F
:101E0800F00000007411F000000090E61A7409F068
:101E180000000012317F90E1C4EFF0E0FF444090F1
:101E28002CE2F0EF541FB42000400302203A901E29
:101E38003DF8282873021E9D021EA8021EB4021E29
:101E4800C0021ECC021EEA021EF6021F02021F0E6C
:101E5800021F1A021F28021F36021F44021F5202C5
:101E68001F60021F6E021F7C021F8A021F98021F3A
:101E7800A6021FB4021FC2021FCF021FDC021FE905
:101E8800021FF602200302201002201D02202A024F
:101E9800203A021EDC7A1979B6122256FD02203544
:101EA8007A1979BC12229D7D010220357A1979C2EE
:101EB8001222567D020220357A1979C812229D7D98
:101EC800030220357BFF7A1979CDE4F53CF53D7D99
:101ED800040220357BFF7A1979D31222587D050236
:101EE80020357A1979D91220F27D080220357A191D
:101EF80079E01220E97D090220357A1979E7122064
:101F0800F27D0A0220357A1979EE1220E97D0B025A
:101F180020357BFF7A1979F41220EB7D0C022035ED
:101F28007BFF7A1979FB1220F47D100220357BFFA4
:101F38007A1A79011220EB7D110220357BFF7A1A7B
:101F480079071220F47D120220357BFF7A1A790D69
:101F58001220EB7D130220357BFF7A1A79121220AA
:101F6800EB7D140220357BFF7A1A79181220F47D54
:101F7800100220357BFF7A1A791E1220EB7D1102A0
:101F880020357BFF7A1A79241220F47D120220353D
:101F98007BFF7A1A792A1220EB7D130220357BFF0A
:101FA8007A1A792F1220EB7D140220357BFF7A1ADA
:101FB80079351220F47D100220357BFF7A1A793B9F
:101FC8001220EB7D1180667BFF7A1A79411220F48A
:101FD8007D1280597BFF7A1A79471220EB7D138096
:101FE8004C7BFF7A1A794C1220EB7D14803F7BFFE3
:101FF8007A1A79521220F47D1080327BFF7A1A798E
:10200800591220EB7D1180257BFF7A1A7960122006
:10201800F47D1280187BFF7A1A79671220EB7D1302
:10202800800B7BFF7A1A796D1220EB7D14123E77B4
:1020380080097BFF7A1A7974122D6CE4FF74C82F1B
:10204800F582E434E1F583E4F02F1222A5E4F00FE1
:10205800BF15EA90401DE4F0123A19C20D123DEC8A
:1020680090E6C37480F090E6C214F000000090E699
:10207800E27402F043B202D21675110112000E90FA
:102088004019E4F090E65EE04438F0E044C4F074AF
:07209800011221480227613B
:1029B800E58070047F0180027F00EF90E68030E0C0
:1029C80006E04408F08004E054F7F0123975300B43
:1029D8002D90401FE030E026C20B7BFF7A1A797BEE
:1029E8001238BD90401FE4F090E6F574FFF0C2097C
:1029F80012225FE4F0000000123E9E123F6C300B82
:102A080059E5BB30E7547BFF7A1A797D1238BD004F
:102A1800000090E6AFE090E6B0122194FED3EF9468
:102A280000EE94004016D390E19BE09F90E19AE07D
:102A38009E400990E6487406F0000000123D417B74
:102A4800FF7A1A79971238BD90E698E0FF123D7D1B
:0D2A580090E699E0FF123D7DC20B023EF6B4
:102A6500E4FF90E6B8E020E703022B0B0F0F74405C
:102A750024011220B6740AF00F744024021220B605
:102A8500E4F00F744024031220B67415F00F74405F
:102A950024041220B67401F00F744024051220B6E8
:102AA5007402F00F744024061220B6E4F00F74404F
:102AB50024071220B67404F00F744024081220B6BF
:102AC500E4F00F744024091220B6E4F00F7440249A
:102AD5000A1220B6E4F00F7440240B1220B6E4F07D
:102AE5000F7440240C1220B6E4F00F7440240D122C
:102AF50020B6E4F00F7440240E1220B6E4F090E7FF
:062B050040EFF01220C7B2
:012B0B0022A7
:102B0C00E4FF9040117404F0A374F0F0A37401F08E
:102B1C00E490E6CEF000000090E6CFF000000090CC
:102B2C00E6D0F000000090E6D17420F000000075B3
:102B3C00BB06000000904019E4F01FEF600AE5BBF3
:102B4C0020E70500000080F2E4FDFCEDAE04780205
:102B5C00C333CE33CED8F92402F58274F81222ADE9
:102B6C001221D1EBF0EDAE047802C333CE33CED8C4
:102B7C00F92403F58274F81222ADFE1222CDEBF08B
:102B8C000DBD00010CED64104C70C0123E9E122164
:102B9C00C890E1DAE0904012F090E1DBE090401355
:012BAC00F038
:012BAD002205
:10338A00E4FF9040117404F0904013E4F090401E62
:10339A007481F0E490E6CEF000000090E6CFF000F1
:1033AA00000090E6D0F000000090E6BEE0C3139063
:1033BA00E6D1F075BB06000000904019E4F01FEF5B
:1033CA00600AE5BB20E70500000080F2E4FF90E612
:1033DA00BEE0FEEFC39E50081220B3E4F00F80EE69
:0333EA00023E9E02
:1030250090E6B8E030E74D90E6BFE0FE90E6BEE002
:10303500FDED4E7002803890E6BDE0705D90E6BC17
:10304500E0147056754EFF754F1A755099755100FD
:1030550075521E7B017AE779411237067B017AE7C3
:103065007940123E62EF0490E740F090E6BEE090B2
:10307500E68BF02290E6BFE0FF90E6BEE04F601AD7
:1030850090E6BFE0701412218D700FEF24BF700A17
:0A30950090E6BEE0B40503123AE431
:01309F00220E
:10005600E4F541F54275110190E6B9E01214200568
:10006600581005581105941204592004B22104BDF4
:100076002204CC2300C32E07B23507AC3801E83979
:1000860000C93C0D313F0853910A3DA20A3DA30A1F
:1000960030A909FDAC00CFB20B6FB301D4B60CFB8F
:1000A600B70886BA08C2BB0230BC05C4BE07CEBFBD
:1000B60001D6C305C4D20106D400000D3612283875
:1000C600020D38123025020D389040117414F012CA
:1000D60022F790E6BCE0905002F090E6BDE090502A
:1000E60002F090E6BAE0905001F090E6BBE0905046
:1000F60001F0D20290E6587410F090E65A0208DC3D
:1001060090E6B8E020E71A90E6A0E020E1F990E753
:1001160040E0FF90E6BCE0FEE42E1222A5EF0205C9
:100126008CE4F53FF540A20233FF1220C0700205B1
:100136003F1222B9F090E65C1220BE7002053F1213
:10014600209F90E65A1220BE7002053F12209F9013
:10015600E65B1220BE7002053F12209F90E6581201
:1001660020BE7002053F12209F90E6591220BE70F5
:1001760002053F12209F90E65E1220BE7002053FE8
:1001860012209F90E65F1220BE7002053F12209F4C
:10019600E4F53DF53E122276C333CE33CED8F912BE
:1001A60020D5FF121022AD07122276C333CE33CEEE
:1001B600D8F92540FFE53F3E1221D1EDF0053EE599
:1001C6003E7002053D6408453D70CA020CF6800C7F
:1001D600122161FD90E6BAE0FB122FA5122B0C024C
:1001E600087790E6B8E020E7307A1A79B0120D6306
:1001F6007BFF60067A1A79BD80047A1A79CA1238AA
:10020600BD90E6BCE0600A146003020D38D20D8092
:1002160002C20D123E06020D3890E6BCE0FFE42F46
:100226001222A5E090E74002058C90E6B8E030E7A0
:100236000302035FE4F510041221487A1A79CF12FB
:100246000D59D39400400A1220C790E6A0E020E1A1
:10025600F990E6BEE0C39404405090E740E030E2F7
:10026600297BFF7A1A79DD1238BD90E743E07BFFE0
:1002760030E0067A1A79EB80047A1A79F71238BDDB
:1002860090E743E013920D123E0690E740E030E11E
:10029600197BFF7A1B79001238BD90E742E0FF1206
:1002A6003D7D90E742E090401FF090E6BEE0600A98
:1002B60090E740E020E0030203547BFF7A1B7912AB
:1002C6001238BD90E6BBE0FF123D7D90E6BAE0FF36
:1002D600123D7D90E6BDE0FF123D7D90E6BCE0FF5D
:1002E600123D7DE5BB30E766E5AC20E06112216199
:1002F6004FFF90E6BDE04FFF90E6BAE04F7003D3A4
:100306008001C392097BFF7A1B79201238BDA209AE
:10031600E433FF123D7D90E6BBE090E6CEF00000B0
:100326000090E6BAE090E6CFF000000090E6BDE06F
:1003360090E6D0F0000000A209E433FF90E6BCE0AE
:100346004F90E6D1F000000075BB060000001222B7
:100356006F1238BDD20B020D38E4F53FF54090E63A
:10036600B01220BE7002053F12209F00000090E6EA
:10037600AF1220BE7002053F12209F00000090E6DB
:10038600991220BE7002053F12209F00000090E6E1
:10039600981220BE7002053F12209F000000E51053
:1003A6005401FF90E6F4E054FE4F1220BF700205A0
:1003B6003F12209F00000090E6141220BE70020536
:1003C6003F12209F00000090E61A1220BE70020520
:1003D6003F12209F00000090E6351220BE700205F5
:1003E6003F12209F00000090E6341220BE700205E6
:1003F6003F12209F0000000540E540AE3F70020519
:100406003F1424401221D5E5ACF000000090E6A987
:100416001220BE7002053F12209F00000090E65495
:100426001220BE7002053F12209F00000090E65584
:100436001220BE7002053F12209F000000300A0401
:100446007F0180027F001220C07002053F1222B990
:1004560002058C7A1B7932120D59B4020E90E6BB56
:10046600E0C4333354C0122132802690E6BEE064E5
:1004760003701E90E6BBE0FF7401A807088002C364
:1004860033D8FC25E044C01221321220FB90E7420B
:10049600F01220FB90E740F090E6BAE075F008A471
:1004A600FFA3E012210890E74102087E7A1B793DFE
:1004B600120D47F0020D387BFF7A1B79481238BDC2
:1004C600E490E68B802490E6B8E030E703020D382E
:1004D60090E6BFE070047F0180027F0090E6BEE0F8
:1004E6004F60347A1B7954120D47F0122161C41300
:1004F6001354037C005403FDE42DF582EC122141D4
:1005060090E6BD122164C413135403FDE42DF58255
:10051600EC122141020D381220C790E6A0E020E13E
:10052600F990E6BEE064046003020D381222F790EB
:10053600E742E0905002F090E743E0905002F090DE
:10054600E740E0905001F090E741E0905001F00262
:100556000D3890E6B8E020E7157BFF7A1B79631229
:1005660038BD1220C790E6A0E020E1F9803D7BFF70
:100576007A1B79721238BD904015E090E740F090F2
:100586004016E090E741F0E490E68A02087E7BFFA1
:100596007A1B79811238BD1220C790E6A0E020E1CF
:1005A600F990E742E05403904014F090E740E09061
:1005B6004015F090E741E0904016F0020D3890E6C5
:1005C600B8E030E7030206F97BFF7A1B799212380E
:1005D600BDC2051220C790E6A0E020E1F990E740F1
:1005E600E090E1C8F0904000F090E741E090E1C96A
:1005F600F0904001F090E742E090E1CAF0904002AE
:10060600F090E743E090E1CBF0904003F090E744B0
:10061600E090E1CCF0904004F090E745E090E1CD29
:10062600F0904005F090E746E090E1CEF09040066D
:10063600F090E747E090E1CFF0904007F090E74870
:10064600E090E1D0F0904008F090E749E090E1D1E9
:10065600F0904009F090E74AE090E1D2F090400A2D
:10066600F090E74BE090E1D3F090400BF090E74C30
:10067600E090E1D4F090400CF090E74DE090E1D5A9
:10068600F090400DF090E74EE090E1D6F090400EED
:10069600F090E74FE090E1D7F090400FF090E750F0
:1006A600E090E1D8F0904010F090E751E090E1D969
:1006B600F0904011F090E752E090E1DAF0904012AD
:1006C600F090E753E090E1DBF0904013F090E1C446
:1006D600E0541FFFD394045003020D38EF641F70DB
:1006E60003020D3890E754E090E1DCF090401DF0F5
:1006F600020D387BFF7A1B79A31238BD90E1C8E062
:1007060090E740F090E1C9E090E741F090E1CAE05F
:1007160090E742F090E1CBE090E743F090E1CCE047
:1007260090E744F090E1CDE090E745F090E1CEE02F
:1007360090E746F090E1CFE090E747F090E1D0E017
:1007460090E748F090E1D1E090E749F090E1D2E0FF
:1007560090E74AF090E1D3E090E74BF090E1D4E0E7
:1007660090E74CF090E1D5E090E74DF090E1D6E0CF
:1007760090E74EF090E1D7E090E74FF090E1D8E0B7
:1007860090E750F090E1D9E090E751F090E1DAE09F
:1007960090E752F090E1DBE090E753F090E1DCE087
:1007A60090E75402087E90E6F574FFF090E6BCE010
:1007B600601090E6AFE090E698F090E6B0E090E644
:1007C60099F0123E9E020D387BFF7A1B79B31238E0
:1007D600BD90E6BEE070277BFF7A1B79C81238BD54
:1007E600904018E0FF123D7D904017E0FF123D7DDE
:1007F60012226F1238BD904019E4F0020D0E90E6F9
:10080600BEE064047BFF702D7A1B79E01238BD9040
:100816004019E4F012220A904019E4F0904017E0E3
:1008260090E742F0904018E090E743F090E68B7432
:1008360004F0020D387A1B79F81238BD12220A909C
:10084600E68B7402F0904019E4F0020D387BFF7AD3
:100856001C79151238BD90E19DE0FF90E740F0EF5E
:100866007BFF70067A1C792280047A1C7929120D86
:100876003A90E6BFE090E68AF090E6BEE0020D0E02
:100886007BFF7A1C79301238BD90E1DDE0FFB401C0
:100896000890E74074BBF0800890E1C4E090E74020
:1008A600F0EF7BFFB401067A1C793D80047A1C794F
:1008B6004A120D3A12212904F0020D3890E6B8E0EA
:1008C60030E71990E6BEE0B4011290E7407401F0FB
:1008D600123A1990E68B7401F0020D387BFF200561
:1008E600107A1C79581238BDD205C20D123DEC8023
:1008F600077A1C79661238BD90E1DDE06401600379
:100906000209DF123DD190E74074BBF090E6BBE0F0
:10091600C313FFE5B154802FF5B1E090E6C4F09023
:10092600E6BAE090E6C5F012218D90E1A0F0A3EFC3
:10093600F090E1A0E0FEA3E0FF4E70030209F0E5AF
:10094600BB30E7EDE5AB20E1E890E19AE0FCA3E0FF
:10095600FDD3EF9DEE9C402290E19AE0FAA3E0FBE6
:10096600EA90E6D0F0000000EB90E6D1F00000003F
:1009760090E156ECF0A3EDF0802790E1A0E0FCA317
:10098600E0FDEC90E6D0F0000000ED90E6D1F0003E
:10099600000090E1A0E0FFA3E090E156CFF0A3EFC6
:1009A600F0E4F5BB000000E5BB20E7030080F8009B
:1009B6000000000090E156E0FEA3E0FFC390E1A135
:1009C600E09FF090E1A0E09EF0E5B1547F04FFE5E2
:1009D600B154802FF5B10209377BFF7A1C79681272
:1009E60038BD90E1C4E090E740F012000E90E6BFFB
:1009F600E012222D020D0E7BFF7A1C79761238BD8D
:100A06007BFF7A1C79851238BD90E6B5E054FEF07E
:100A160090E6BFE01220C890E6BBE090E6B3F09007
:100A2600E6BAE090E6B4F0020D3890E1C67401F043
:100A360090E159E04401F07BFF7A1C79931238BDAE
:100A460090E6BAE0753700F538A3E0FEEE4237903F
:100A5600E6BEE0753900F53AA3E0FEEE423990E6CF
:100A6600B8E064C06003020B10E53A453970030232
:100A76000D3890E6A0E020E1F9C3E53A9440E53967
:100A86009400500885393B853A3C8006753B0075D5
:100A96003C4090E6B9E064A3704090E6BCE0B40147
:100AA6001BA3E0701790E6BBE030E71090E74074B8
:100AB60003F0A37401F0A37407F08042E4F53DF55A
:100AC6003E122222503812227DE0FF1221B9EFF0A9
:100AD600053EE53E70EB053D80E7E4F53DF53E124B
:100AE600222250101221B974CDF0053EE53E70EF7A
:100AF600053D80EB122119AF38AE37123758122157
:100B060029E53CF0122175020A6F90E6B8E06440D0
:100B16006003020D38E53A45397003020D3812219B
:100B260029F090E6A0E020E1F990E68BE0753B0025
:100B3600F53C90E6B9E0B4A31EE4F53DF53E12227D
:100B460022501E1221B9E0FF12227DEFF0053EE58C
:100B56003E70EB053D80E7122119AF38AE371239EA
:100B6600E4E53C122175020B1B90E6B8E030E70382
:030B7600020C1E50
:100B790090E6BDE030E60312276190E6BDE030E77C
:100B890004C2068004A201920690E6BEE0701B7BB7
:100B9900FF7A1C79A91238BD1220CC122161FD906F
:100BA900E6BAE0FB122FA5020D387BFF7A1C79BC4F
:100BB9001238BD1220C790E6A0E020E1F9E4F53D26
:100BC900F53E90E740E0F543E5437003020D38C375
:100BD900E53E9404E53D94004003020D38E54330B9
:100BE900E023AF3EC007E53E25E0FFE53D33FE7457
:100BF900422FF58274E73EF583E0FD1222CDE0FB3A
:100C0900D007122FA5053EE53E7002053DE543C319
:050C190013F54380B358
:100C1E007A1C79D4120D636076754BFF754C1C757A
:100C2E004DE690E1A41220DEF5518E508D4F8C4E84
:100C3E00A31220DEF5558E548D538C52A31220DE56
:100C4E00F5598E588D578C56A31220DEF55D8E5CAD
:100C5E008D5B8C5AA31220DEF5618E608D5F8C5EEB
:100C6E00A31220DEF5658E648D638C62A31220DEE6
:100C7E00F5698E688D678C66A31220DEF56D8E6C1D
:100C8E008D6B8C6A7B017AE779401215778059A2B9
:100C9E0001E43390E740F0A206E433A3F0E4A3F0BE
:100CAE00A3F0F53DF53E122276C333CE33CED8F9FE
:100CBE001220D5FFC004C005C006C007122276C39D
:100CCE0033CE33CED8F92444F58274E73EF583D083
:100CDE0007D006D005D0041213D3053EE53E7002B0
:100CEE00053D6408453D70BE12222C80137BFF7AB1
:100CFE001D79201238BD90E6B8E030E70912222C9B
:100D0E0090E68BF0802490E6BEE0D394004005E0A0
:100D1E0090E68BF090E19CE0448090401EF01238FB
:0B0D2E00FD8007122A658002D322C35B
:100D3900221238BD7BFF7A19799A1238BD227BFFBE
:100D49001238BDE490E68BF090E6BBE090500322A8
:100D59007BFF1238BD90E6BEE0227BFF1238BD90C2
:040D6900E6BCE022E2
:103EC2007BFF7A1D79331238BD7F017E001237F2F3
:023ED200D322F9
:103ED4007F017E001237F27BFF7A1D79411238BDD3
:023EE400D322E7
:023F7600D32254
:1036030090E680E030E72100000090E6247402F0A9
:10361300000000E490E625F0000000D20790E19A54
:103623007402F0A3E4F0801F000000E490E624F0AD
:1036330000000090E6257440F0000000C20790E10E
:103643009AE4F0A37440F090E6BAE090E1C5F0127A
:07365300226F1238BDD322E3
:0A3F2B0090E1C512212404F0D32216
:0A3F350090E6BAE090E158F0D322C4
:0A3F3F0090E15812212404F0D3226F
:023F7800D32252
:023F7A00D32250
:023F7C00D3224E
:103C5F00C0E0C083C082C085C084C086758600D294
:103C6F001712216E7401F0D086D084D085D082D007
:043C7F0083D0E032DC
:103CC600C0E0C083C082C085C084C08612216B74E8
:0F3CD60004F0D086D084D085D082D083D0E03265
:103CE500C0E0C083C082C085C084C08612216B74C9
:0F3CF50002F0D086D084D085D082D083D0E03248
:1032BB00C0E0C0F0C083C082C085C084C086758664
:1032CB0000C0D075D000C000C001C002C003C00454
:1032DB00C005C006C007856D69856E6A1222D88548
:1032EB00656B85666C1222E312216E7410F07BFF06
:1032FB007A1D794E123252D007D006D005D004D0A9
:10330B0003D002D001D000D0D0D086D084D085D0CD
:08331B0082D083D0F0D0E03233
:103D0400C0E0C083C082C085C084C08612216B74A9
:0F3D140008F0D086D084D085D082D083D0E03222
:10393A00C0E0C083C082C085C084C08675860090FE
:10394A00E680E030E71285656985666A1222D885C5
:10395A006D6B856E6C1222E312216E7420F0D08694
:0B396A00D084D085D082D083D0E03222
:013F7E003210
:013F7F00320F
:013F8000320E
:013F8100320D
:103C8300C0E0C083C082C085C084C0867586001230
:103C9300228A7404F0D086D084D085D082D083D099
:023CA300E0320D
:102F1C00C0E0C0F0C083C082C085C084C086758606
:102F2C0000C0D075D000C000C001C002C003C004F6
:062F3C00C005C006C0073D
:102F420090E68DE0FF90E6A2E020E127E4FEEEC3EA
:102F52009F501B74802EF582E434E7F583E0FD7404
:102F6200C02EF582E434E7F583EDF00E80E090E6C2
:102F72008FEFF07BFF7A1D795612325212228A7439
:022F820008F055
:102F8400D007D006D005D004D003D002D001D000A1
:102F9400D0D0D086D084D085D082D083D0F0D0E079
:012FA40032FA
:10365A00C0E0C0F0C083C082C085C084C0867586C1
:10366A0000C0D075D000C000C001C002C003C004B1
:10367A00C005C006C0077BFF7A1D795C1232521260
:10368A00228A7410F0D007D006D005D004D003D017
:10369A0002D001D000D0D0D086D084D085D082D0BC
:0636AA0083D0F0D0E032F5
:013F8200320C
:1036B000C0E0C0F0C083C082C085C084C08675866B
:1036C00000C0D075D000C000C001C002C003C0045B
:1036D000C005C006C0077BFF7A1D79641232521202
:1036E000228A7440F0D007D006D005D004D003D091
:1036F00002D001D000D0D0D086D084D085D082D066
:0637000083D0F0D0E0329E
:013F8300320B
:1030A000C0E0C0F0C083C082C085C084C086758681
:1030B00000C0D075D000C000C001C002C003C00471
:0630C000C005C006C007B8
:1030C6005391EF75100190E659E0F524300205C2E0
:1030D600021221C87BFF7A1D796D12325290E65991
:0930E60074FFF090E65B7401F048
:1030EF00D007D006D005D004D003D002D001D00035
:1030FF00D0D0D086D084D085D082D083D0F0D0E00D
:01310F00328D
:013F8400320A
:013F85003209
:1033ED00C0E0C0F0C083C082C085C084C086758631
:1033FD0000C0D075D000C000C001C002C003C00421
:10340D00C005C006C0075391EF90E65B7410F07BCA
:10341D00FF7A1D7971123252D007D006D005D00433
:10342D00D003D002D001D000D0D0D086D084D085AA
:09343D00D082D083D0F0D0E0323F
:013F86003208
:10344600C0E0C0F0C083C082C085C084C0867586D7
:1034560000C0D075D000C000C001C002C003C004C7
:10346600C005C006C0075391EF90E65B7440F07B41
:10347600FF7A1D7974123252D007D006D005D004D7
:10348600D003D002D001D000D0D0D086D084D08551
:09349600D082D083D0F0D0E032E6
:013F87003207
:013F88003206
:013F89003205
:013F8A003204
:013F8B003203
:013F8C003202
:013F8D003201
:013F8E003200
:013F8F0032FF
:013F900032FE
:10349F00C0E0C0F0C083C082C085C084C08675867E
:1034AF0000C0D075D000C000C001C002C003C0046E
:1034BF00C005C006C0075391EF90E6517402F07B30
:1034CF00FF7A1D7978123252D007D006D005D0047A
:1034DF00D003D002D001D000D0D0D086D084D085F8
:0934EF00D082D083D0F0D0E0328D
:013F910032FD
:1034F800C0E0C0F0C083C082C085C084C086758625
:1035080000C0D075D000C000C001C002C003C00414
:10351800C005C006C0075391EF90E6557402F07BD2
:10352800FF7A1D797C123252D007D006D005D0041C
:10353800D003D002D001D000D0D0D086D084D0859E
:09354800D082D083D0F0D0E03233
:013F920032FC
:10355100C0E0C0F0C083C082C085C084C0867586CB
:1035610000C0D075D000C000C001C002C003C004BB
:10357100C005C006C0075391EF90E6517401F07B7E
:10358100FF7A1D7980123252D007D006D005D004BF
:10359100D003D002D001D000D0D0D086D084D08545
:0935A100D082D083D0F0D0E032DA
:013F930032FB
:1035AA00C0E0C0F0C083C082C085C084C086758672
:1035BA0000C0D075D000C000C001C002C003C00462
:1035CA00C005C006C0075391EF90E6557401F07B21
:1035DA00FF7A1D7984123252D007D006D005D00462
:1035EA00D003D002D001D000D0D0D086D084D085EC
:0935FA00D082D083D0F0D0E03281
:013F940032FA
:013F950032F9
:013F960032F8
:06383800AB07AA06AC0577
:10383E00E4FD90E1C6E0600B7E000DEE24DE122268
:10384E00C5EAF0AE050D74DE2E1222C5EBF0AF0503
:10385E000D74DE2F1222C5ECF090E159E0FF7AE1F3
:0D386E007BDE123DB590E159E0FF0239AE5E
:0A39E4008E448F458D468A478B48BC
:1039EE00E4F549E549C3954650200545E545AE4405
:1039FE007002054414FFE5482549F582E43547F584
:0A3A0E0083E0FD123838054980D925
:013A1800228B
:0A3758008E468F478D488A498B4A40
:10376200E4FDF54B90E1C6E06012E546FF7E000DF8
:10377200EE24DEF582E434E1F583EFF0AE050D745C
:10378200DE2EF582E434E1F583E547F090E159E07D
:10379200FF7AE17BDE123DB590E159E0FFAB4AAA28
:0637A20049AD48023D990B
:103DEC00A20D920A90401F300A07E4F0122C438077
:0A3DFC00067402F0122BAE023E9E88
:103E0600A20D920A90401F300A07E4F0122C43805C
:0A3E1600067402F0122BAE023E9E6D
:10332300EFC3940250047E0E80027E0FAB06EF546F
:1033330001FE90E67AE04401F0C2E990E678E044C9
:1033430080F0EB25E090E679F090E678E030E0F964
:10335300EE441890E679F090E678E030E0F9EC90EE
:10336300E679F090E678E030E0F9ED90E679F090D8
:10337300E678E04440F090E678E030E0F990E678D3
:06338300E020E6F9D2E9AA
:013389002221
:093F5B00050DE50D7002050C22B4
:08000300E4F51ED2E9D2AF22A0
:1039AE0090E678E020E6F9C2E990E678E04480F00F
:1039BE00EF25E090E679F090E678E030E0F990E6D9
:1039CE0078E04440F090E678E020E6F990E678E082
:0639DE0030E1D6D2E9221F
:103A8100A90790E678E020E6F9E51E702390E67834
:103A9100E04480F0E925E090E679F08D19AF03A9C3
:103AA10007751A018A1B891CE4F51D751E01D322B5
:023AB100C3222E
:103A4D00A90790E678E020E6F9E51E702590E67866
:103A5D00E04480F0E925E0440190E679F08D19AF5E
:103A6D0003A907751A018A1B891CE4F51D751E0330
:043A7D00D322C3226B
:03004B0002265931
:10265900C0E0C083C082C085C084C086758600C0C2
:10266900D075D000C000C001C002C003C006C007B9
:1026790090E678E030E206751E0602274390E67878
:10268900E020E10CE51E64026006751E070227437F
:10269900E51E24FE605F14603624FE7003022734B1
:1026A90024FC700302274024086003022743AB1A65
:1026B900AA1BA91CAF1D051D8F827583001212FE6E
:1026C90090E679F0E51D65197070751E05806B90AF
:1026D900E679E0AB1AAA1BA91CAE1D8E8275830090
:1026E90012133D751E02E5196401704E90E678E0FB
:1026F9004420F08045E51924FEB51D0790E678E0F1
:102709004420F0E51914B51D0A90E678E04440F03C
:10271900751E0090E679E0AB1AAA1BA91CAE1D8EA6
:102729008275830012133D051D800F90E678E04401
:1027390040F0751E008003751E005391DFD007D04D
:1027490006D003D002D001D000D0D0D086D084D01A
:0827590085D082D083D0E0326C
:103D9900123A4DE51E24FA600E146006240770F3EA
:0C3DA900D322E4F51ED322E4F51ED32241
:103DB500123A81E51E24FA600E146006240770F39A
:0C3DC500D322E4F51ED322E4F51ED32225
:100D6D0002108EE86480F8E933E83360110460F016
:100D7D00ED33EC337009E8FCE9FDEAFEEBFF2204EC
:100D8D0060DED3EB9FEA9EE99DE8C2E78CF0C2F7E7
:100D9D0095F0400CE8CCF8E9CDF9EACEFAEBCFFBB3
:100DAD0012105985D0F05804700320D5B3E80470A3
:100DBD00075002B2D502109892D5EC0460F7E4CC3E
:100DCD00C0E0C398F8603B94186008400DD0E0FB7C
:100DDD00021070E4FBFAC9FC8028E830E406E4C98F
:100DED00FBE4CAFCE830E305E4C9CACBFCE85407D0
:100DFD006010F8C3E913F9EA13FAEB13FBEC13FCDB
:100E0D00D8F130F52FC3E49CFCEF9BFFEE9AFEED7D
:100E1D0099FDD0E0FBEF4E4D4C701222DB0302101A
:100E2D0095EC2CFCEF33FFEE33FEED33FDED30E7AB
:100E3D00EB021070EF2BFFEE3AFEED39FDD0E0FB2B
:100E4D0050130BBB0003021098ED13FDEE13FEEFD4
:080E5D0013FFEC13FC021070FE
:100E6500EC4D6011E8497017ED33EC3304600DE487
:100E7500FCFFFEFD22E933E8330470F802108E1200
:100E8500105958046009E4CC248150062850090201
:100E95001098284003021095C0E0EB4A7044B980D1
:100EA50006D0E0FB021084EF4E701CBD8008EBFFFE
:100EB500EAFEE9FD80EBE98DF0A4FEE5F0020F4EB8
:100EC500E9CDF9EAFEEBFFEF89F0A4FCE5F0CE8968
:100ED500F0A42EFFE435F0CD89F0A42DFEE435F025
:100EE5008067EF4E7005BD80D780C3EF8BF0A4AC53
:100EF500F0EE8BF0A42CFCE435F0F8EF8AF0A42C8E
:100F0500E5F038FCE433CB8DF0A42CFCE5F03BF8A0
:100F1500EE8AF0A42CFCE5F038F8E433CF89F0A490
:100F25002CFCE5F038CF3400CE89F0A42FFFE5F096
:100F35003EFEE433C98DF0A42EFEE5F039CD8AF0EE
:100F4500A42FFFE5F03EFEE43DFD33D0E0FB500766
:100F55000BBB000F021098EC2CFCEF33FFEE33FEB9
:060F6500ED33FD021070E7
:100F6B0074F8CC6480CCC86480C8F58204604FC32D
:100F7B00EB9FF5F0EA9E42F0E99D42F0E89C45F0CC
:100F8B00603C501DE5825FFFE582D313CB5BCBF456
:100F9B002B5582FB50280ABA002409B9002008807F
:100FAB001DE5825BFBE582D313CF5FCFF4C3132F19
:100FBB005582FF50090EBE00050DBD00010CC3EBA1
:100FCB009FF5F0EA9E42F0E99D42F0E89C45F06007
:090FDB0007CC4820E701B3EC2229
:100FE40075F020800E75F010800575F0087D007E88
:100FF400007F003392D530D5031213B4EC33401084
:10100400EF33FFEE33FEED33FDEC33FCD5F0ED2290
:0E101400E5F0247EA2D513CC92E7CDCEFF22CC
:10102200EDD2E7CD33EC3392D524814006E4FFFEC6
:10103200FDFC22FCE4CFCECDCC24E0501174FF8025
:10104200EDC3CC13CCCD13CDCE13CECF13CF0470C2
:07105200F030D5DE0213B4FB
:10151B00E55F244BF8E6055F227848301402784BE0
:10152B00E475F0011214100212E5200DEB7F2ED2A0
:10153B000D8018EF540F2490D43440D4FF30110B8E
:10154B00EF24BFB41A0050032461FFE5606002155D
:10155B00600563E5637002056230140D7848E4752D
:10156B00F001121410EF02132B023BEE7403D21492
:10157B008003E4C214F55F8B488A49894AE4F5601D
:10158B00F562F563E56060077F2012155680F575EF
:10159B0061FFC20EC20DC20FC210C212C213C2151E
:1015AB00121524FF700D3014057F00121567AF6301
:1015BB00AE6222B4255FC2D5C211121524FF24D00E
:1015CB00B40A00501A75F00A786030D50508B6FFDA
:1015DB000106C6A426F620D5047002D21080D924A9
:1015EB00CFB41A00EF5004C2E5D211021854D20E38
:1015FB0080C6D20D80C0D20F80BCD2D580BAD21299
:10160B0080B47F20121556200F077401B56000407F
:10161B00F112151BFF12155602158FD215D213801E
:10162B009512151BFB12151BFA12151BF94A4B7061
:10163B0006794B7A197BFF200F2EE560602A7E001E
:10164B008E827583001212FE60060EEE656170F0DD
:10165B00C2D5EBC0E0EAC0E0E9C0E0EE1218B4D0AE
:10166B00E0F9D0E0FAD0E0FB1212E5FF60AAEBC084
:10167B00E0EAC0E0E9C0E0121556D0E02401F9D051
:10168B00E03400FAD0E0FBE5610460DCD561D98081
:10169B0087D20F80A212189760F7E56170010412D0
:1016AB0010A3A961600DE561600914F56112193E83
:1016BB00EF60F3EA30E702F404C3995077EAF425BC
:1016CB00610430E701E404F561800D12189760C1E5
:1016DB00EA056125611210A3EA785EF630E701E4B2
:1016EB00256104D56104201201141218B4E4C0E082
:1016FB0012193E785EE6601320E70714F612153ECA
:10170B00802204F6D0E014C0E07F0012153EE561A4
:10171B0060071215351561800B301203121535D089
:10172B00E002158FD0E00480C512189760A0E56128
:10173B00041210A3785EEAF6E56120120260010440
:05174B0024041218B493
:1017500074FF04C0E012193E12153EE5612012022A
:101760006003121535D0E0B561E87F451215487861
:101770005EE67F2B30E7047F2DF404C0E01215569F
:10178000D0E075F00A84C0F012153FD0E012153F8A
:1017900002158F791080027908C213C2158008D211
:1017A000D5790A8004790AC2D5E561047002F56131
:1017B000E4FAFDFEFF12151BFC7B08200E13121528
:1017C0001BFD7B10300D0A12151BFE12151BFF7B33
:1017D00020EC3382D592D55013C3E4300D069FFF21
:1017E000E49EFEE4200E039DFDE49CFCE4CBF8C2E5
:1017F0000EEC700CCFCECDCCE824F8F870F3801747
:10180000C3EF33FFEE33FEED33FDEC33FCEB33FB84
:10181000994002FB0FD8E9EB300E05F8D0E0C44840
:10182000B20EC0E00AEC4D4E4F78207B0070C2EA49
:10183000B5610040BCC0E01218B6D0F0D0E0200E78
:1018400004C4C0E0C4B20EC0F012153FD0F0D5F011
:10185000EB02158F121420162C5317935815FD4CBC
:1018600015F94217974F179F44179F4916124317B0
:10187000A55516D64617344516A047196B501601C4
:101880002D16052E16282B16092316262019542A44
:1018900015C14800001620E561B4FF03756106120A
:1018A000151BFC12151BFD12151BFE12151BFF78D4
:1018B000570210D2790AA2D5201014301209B9109B
:1018C000020404B9080104A2D52013025001042027
:1018D0000F68920FB560005034C0E07F20301019BF
:1018E0007F30A20F72137212500F12190DC20FC265
:1018F00013C212C2157F30800F301203E9C0E0120C
:101900001556301203D0E0F9D0E0B560CC30121794
:101910007F30B9100C1215567F583011077F788030
:1019200003B90803121556300F057F2D0215567F97
:10193000202015F87F2B2013F322920F80CF7F00F9
:10194000B4070050052457F8E6FF22286E756C6C2A
:101950002900D20E12151B300EF8C20E786030D559
:101960000108F60215C12D5043495812151B2403D6
:10197000B405004001E490196693121547743A12B9
:0A1980001547D2107560040217939A
:10105900E9D2E7C933E833F892D5EDD2E7CD33ECDD
:0710690033FC5002B2D52256
:10107000EC30E7100FBF000C0EBE00080DBD0004E1
:101080000BEB6014A2D5EB13FCED92E7FD2274FF8D
:10109000FCFDFEFF22E480F8A2D574FF13FC7D80E6
:0310A000E480EFFA
:1010A300F920E72824F950037907E4F42402FB1814
:1010B300DBFDE624FB5014E9600DE4F618E604F6C4
:0F10C300B40A08E4F6D9F57401F60A22C2D52260
:1010D200ED33EC3392D5FA602AB4FF33EDC2E77BED
:1010E200FF60067A1079F7E4227A11790020D5049C
:1010F2007A1079FB224E614E002B494E46002D4953
:101102004E4600E47A08F608DAFC7B00740722E80F
:10111200C0E0ECC0E0EDC0E0EEC0E0EFC0E0EA7598
:10112200F010A4CAABF075F04DA42BFBE435F0FC33
:10113200EA2410FAEB34C5FBEC34D9FCEDC2E7FF2C
:1011420075F056A4F42411C5F0F434C58FF0A42A26
:10115200E5F03BE43CF620E7141212A5D0E0FFD004
:10116200E0FED0E0FDD0E0FC1211D88014F40412AD
:1011720012A5D0E0FFD0E0FED0E0FDD0E0FC120EE0
:1011820065D0E0F8E6FAEDD2E7CD33EC332482FB0A
:10119200E4C3CF33CFCE33CECD33CD33DBF37B07B6
:1011A20075F00A846004F6081B0AE5F0F6088FF071
:1011B200740AA4FFACF08EF0740AA42CFEACF050BA
:1011C200010C8DF0740AA42CFDE435F0F608DBDE88
:0311D2007407227D
:1011D500021098EC5D046005E85904700302108E56
:1011E500121059580460F6EC4860F2EC7004FDFEEC
:1011F500FF22C860DB2481C85009C39860025006ED
:101205000210959850CAF582E9294B4A7005AB82C0
:1012150002108475F0007C1A7880C3EF9BEE9AED7E
:1012250099400DC3EF9BFFEE9AFEED99FDE842F064
:10123500DC23ACF0D0E0FFD0E0FED0E0FDAB8220B7
:10124500E7101BEB60BAEC2CFCEF33FFEE33FEED41
:1012550033FD021070E803F830E705C0F075F000C3
:10126500EF2FFFEE33FEED33FD40B830E7C280AA25
:101275003F8000004120000042C80000447A000081
:10128500461C400047C35000497424004B18968003
:101295004CBEBC205A0E1BCA6753C21C749DC5AEFA
:1012A500FB60065407601C23231212D3EB543860ED
:1012B500091212BF1212CE120E65ECF8EDF9EEFA14
:1012C500EFCB22EB1212CE80F1543803241C90127E
:1012D50075FE93FC0EEE93FD0EEE930ECE93FF225C
:03000000022E903D
:0C2E9000787FE4F6D8FD758177022ED71C
:1012E500BB010689828A83E0225002E722BBFE0207
:0912F500E32289828A83E493223A
:1012FE00BB010CE58229F582E5833AF583E02250A5
:10130E0006E92582F8E622BBFE06E92582F8E222EE
:0D131E00E58229F582E5833AF583E4932208
:10132B00BB010689828A83F0225002F722BBFE01A1
:02133B00F3229B
:10133D00F8BB010DE58229F582E5833AF583E8F0E6
:10134D00225006E92582C8F622BBFE05E92582C892
:02135D00F2227A
:10135F00BC000BBE0029EF8DF084FFADF022E4CC72
:10136F00F875F008EF2FFFEE33FEEC33FCEE9DEC3B
:10137F00984005FCEE9DFE0FD5F0E9E4CEFD22ED81
:10138F00F8F5F0EE8420D21CFEADF075F008EF2FCB
:10139F00FFED33FD4007985006D5F0F222C398FDBC
:0513AF000FD5F0EA2259
:0E13B400C3E49FFFE49EFEE49DFDE49CFC224A
:1013C200EB9FF5F0EA9E42F0E99D42F0E89C45F081
:0113D20022F8
:0C13D300ECF0A3EDF0A3EEF0A3EFF0228D
:1013DF00A8828583F0D083D0821213F61213F612EF
:1013EF0013F61213F6E473E493A3C583C5F0C58314
:1013FF00C8C582C8F0A3C583C5F0C583C8C582C858
:01140F0022BA
:10141000FAE6FB0808E6F925F0F618E6CA3AF622DD
:10142000D083D082F8E4937012740193700DA3A35B
:1014300093F8740193F5828883E47374029368606F
:06144000EFA3A3A380DF6F
:103BEE00EFB40A07740D123BF9740A309811A899B4
:103BFE00B8130CC2983098FDA899C298B811F63037
:073C0E0099FDC299F599220E
:103706008B4B8A4C894DE4F553F554E5521552AE70
:1037160051700215514E6033AB4EAA4FA95012128A
:10372600E5FFAB4BAA4CA94D0554E554AC537002CA
:10373600055314F5828C83EF12133DEF60CD7401AF
:103746002550F550E4354FF54F80C0AB4BAA4CA938
:023756004D2202
:103E6200E4FFFE1212E5600C0FEF70010E09E9701B
:053E7200F20A80EF22BE
:10144600E709F60870FA8046E709F20870FA803E66
:1014560088828C83E709F0A370FA8074E309F608A2
:1014660070FA806CE309F20870FA806488828C83D3
:10147600E309F0A370FA805889828A83E0A3F6080C
:1014860070FA804C89828A83E0A3F20870FA804061
:1014960080D280FA80C680D4805180F28027801066
:1014A60080A680EA809A80A880DA80E280CA8027B7
:1014B60088848C8589828A83E493A30586F0A305B4
:1014C6008670F5800B89828A83E493A3F60870F907
:1014D600ECFAA9F0EDFB2288848C8589828A83E068
:1014E600A30586F0A3058670F680E589828A83E4E3
:1014F60093A3F20870F980D888F0ED2402B40400B2
:1015060050CEF582EB2402B4040050C42323458256
:05151600239014967300
:102E9C00022DFFE493A3F8E493A34003F68001F220
:102EAC0008DFF48029E493A3F85407240CC8C33337
:102EBC00C4540F4420C8834004F456800146F6DF06
:102ECC00E4800B0102040810204080902301E47E72
:102EDC00019360BCA3FF543F30E509541FFEE493FB
:102EEC00A360010ECF54C025E060A840B8E493A3C2
:102EFC00FAE493A3F8E493A3C8C582C8CAC583CAED
:102F0C00F0A3C8C582C8CAC583CADFE9DEE780BEA4
:0124AE00002D
:00000001FF
